S02000006F70656E62746C5F6F6C696D65785F65666D3332673838302E7372656320
S113000070070020C91B0000ED1B0000ED1B000061
S1130010ED1B0000ED1B0000ED1B0000ED1B0000BC
S1130020ED1B0000ED1B0000ED1B0000ED1B0000AC
S1130030ED1B0000ED1B0000ED1B0000ED1B00009C
S1130040ED1B0000ED1B0000ED1B0000ED1B00008C
S1130050ED1B0000ED1B0000ED1B0000ED1B00007C
S1130060ED1B0000ED1B0000ED1B0000ED1B00006C
S1130070ED1B0000ED1B0000ED1B0000ED1B00005C
S1130080ED1B0000ED1B0000ED1B0000ED1B00004C
S1130090ED1B0000ED1B0000ED1B0000ED1B00003C
S11300A0ED1B0000ED1B0000ED1B0000ED1B00002C
S10B00B0ED1B0000ED1B000034
S11300B8890011EB401010F1844002607047DFF8AA
S11300C88405006810F007010029012903D9891E55
S11300D8012904D906E0012161F3020002E00321A9
S11300E861F30200DFF85C1508607047B0FA80F02D
S11300F8D0F11F007047DFF84C150968DFF8482570
S1130108821ADFF848359A420BD211F00702921E80
S1130118012A03D8032262F3020102E0012262F3F6
S11301280201DFF8242590420AD211F00700801E4C
S1130138012803D8022060F3020101E0C908C900BC
S1130148DFF8000501607047DFF80405704780B5E3
S1130158DFF8000500F09EF9C0B2072804D008288B
S113016805D100F0AEFA03E0FFF7EEFF00E000204F
S113017802BD80B5DFF8E0140968C0B2400031FA66
S113018800F010F0030000280FD0022806D002D394
S1130198032806D00BE000F0CEFA09E000F0CEFA0E
S11301A806E000F083FA400802E0002000E00020A6
S11301B802BDDFF8A8140968C90704D4DFF8A0143D
S11301C809680142FAD1704710B50C00C0F3031155
S11301D8012907D0C0F09A80032925D010D3042917
S11301E867D093E02000FFF781FF0400DFF87C0468
S11301F80068000900012043DFF87014086085E0F6
S1130208FFF75DFF2000FFF771FF0400DFF86004CB
S11302180068000900012043DFF85414086000F066
S113022845FAFFF768FF71E0DFF84814884208D000
S1130238DFF84414884215D0DFF84414884223D0E8
S113024836E00420FFF7B5FF2000FFF74FFF040056
S1130258DFF828040068000900012043DFF81C14B3
S1130268086025E00420FFF7A4FF2000FFF73EFF05
S11302780400DFF80804006830F0F00050EA0410C5
S1130288DFF8F813086013E00420FFF792FF20005A
S1130298FFF72CFF0400DFF8E403006830F4407033
S11302A8B4F1100150EA0120DFF8D0130860FFE729
S11302B82CE0DFF8D013884204D0DFF8CC1388424E
S11302C811D022E04020FFF774FF2000FFF70EFF53
S11302D80400DFF8B8030068800880002043DFF8D2
S11302E8AC13086011E04020FFF763FF2000FFF71C
S11302F8FDFE0400DFF89403006830F0300050EA93
S11303080410DFF888130860FFE7FFE710BD70B535
S11303180C000021C0F30322D2B2012A09D029D348
S1130328032A19D015D3052A1DD018D3062A1ED09E
S113033820E0DFF83853C0F30436002902D008005F
S1130348FFF737FFE4B2220031002800FFF7B0FEC0
S113035870BDDFF83C53EEE7DFF83853EBE7DFF81E
S113036838530121E7E7DFF834531021E3E7DFF8D6
S11303783053E0E7ECE780B510F47810002824D077
S1130388B0F5003F24D0B0F5802F2AD0B0F5C02FA7
S11303982AD0B0F5002F2BD0B0F5202F32D0B0F5ED
S11303A8402F39D0B0F5602F41D0B0F5901F51D00F
S11303B8B0F5A01F52D0B0F5B01F59D0B0F5C01F8A
S11303C860D0B0F5D01F60D062E000F07AF960E048
S11303D800F077F9DFF89412096811F00F01C840AA
S11303E857E000F063F954E00020FFF7C2FE50E044
S11303F80020FFF7BEFEDFF88412096811F00F0130
S1130408C84046E00020FFF7B4FEDFF87012096820
S1130418C1F30311C8403CE00020FFF7AAFEDFF84F
S11304285C120968090A11F00301C84031E0002090
S1130438FFF79FFEDFF844120968090A11F0030167
S1130448C840DFF86012096811F00701491CB0FBC5
S1130458F1F01EE00120FFF78CFE1AE00120FFF7FF
S113046888FEDFF82812096811F00301C84010E07B
S11304780120FFF77EFEDFF814120968C1F30111A9
S1130488C84006E0FFF763FE03E0FFF75DFE00E007
S1130498002002BD012110F00F00012806D036D338
S11304A803282DD018D304282FD030E0DFF8B80162
S11304B8006810F47050B0F5006F09D0B0F5805F93
S11304C804D0B0F5005F05D1022104E0032102E065
S11304D8042100E005211BE0DFF87C01006810F02E
S11304E80300012804D009D3032805D002D305E06A
S11304F8032104E0022102E0062100E0012107E0D3
S1130508DFF854010068012102E0072100E000211E
S11305180800C0B2704738B50324032310F00F0055
S11305280200521E03D0521E012A27D956E0C9B22E
S1130538022906D021D3042919D015D3052919D0A5
S11305481BE004240023012201211800C0B200F09A
S113055846F8FFF7B4FD4348046000F00BF900F0D7
S1130568A5F8FFF7C8FD39E003240123EBE70224CB
S11305780223E8E701240323E5E72FE0022801D159
S1130588002400E00224C9B2012906D002290FD0B0
S1130598032914D0062919D01FE000202E49096820
S11305A80322A2409143A04008432B49086015E068
S11305B801220121002000F012F80220EEE70122B6
S11305C80121012000F00BF80120E7E701220221B4
S11305D83048FFF76DFD0320E0E7FFE731BD10B5B4
S11305E8C0B2002821D0022813D01AD3042814D06A
S11305F822D2012302240220C9B200291DD02A498B
S11306080B60D2B2002A1AD017490968014216D1E0
S1130618FAE7042308240820EEE7102320242020E6
S1130628EAE7402380248020E6E74FF480734FF400
S113063800744FF40070DFE703E01B48046000F027
S113064899F810BD04000C400124F4000024F400BF
S1130658809FD5000400180028800C4054800C406A
S113066850800C4024800C402C800C4008800C40A6
S113067804800C403004080030140A0068800C40E0
S113068830000C00400514004015160070800C4022
S113069844800C4040800C4058800C4060800C40E2
S11306A878800C407C800C4020800C4080B500F0A1
S11306B808F82449096811F00F01C8402249086064
S11306C802BD2248006810F47050B0F5006F0BD0DA
S11306D8B0F5805F05D0B0F5005F08D11C4800680C
S11306E827E04FF4004024E01A48006821E01A4843
S11306F8006810F4E060002818D0B0F5807F13D0AB
S1130708B0F5007F0ED0B0F5407F09D0B0F5806F0A
S113071804D0B0F5A06F0BD110480AE0104808E0E7
S1130728104806E0104804E0104802E0104800E0D1
S11307380020704770474FF4004070470448006831
S11307487047000004800C405C0600202C800C409C
S1130758700100206C0100200C800C40003FAB01AC
S1130768406F4001809FD500C0D8A700C0CF6A0061
S113077840420F000248034909680180704700009D
S1130788680600202C800C40DFF800F08900002067
S1130798DFF800F00100002080B500F045FADFF82A
S11307A878045FF0FF310160DFF870045FF0FF3117
S11307B8016001BD70B504000D001600200000F0B2
S11307C8C7F9FF2805D02819401E00F0C1F9FF28F1
S11307D801D1002017E0600A4FF400714843DFF8A4
S11307E840140968884207D12B0032002100DFF841
S11307F82C0400F0EBF806E02B0032002100DFF8AF
S1130808180400F0E3F870BD70B504000D00200072
S113081800F09EF906002819401E00F099F9F6B276
S1130828FF2E02D0C0B2FF2801D1002005E001004C
S1130838C9B23000C0B200F04AF970BD80B50020DA
S11308480090DFF8D803006810F1010F01D10120EE
S113085837E00098DFF8C413496808180090009836
S1130868DFF8B8138968081800900098DFF8AC130B
S1130878C968081800900098DFF8A01309690818D7
S113088800900098DFF894134969081800900098BC
S1130898DFF888138969081800900098DFF87C133A
S11308A8C969081800900098C04300900098401C3B
S11308B8009000AA0421DFF868030068B830FFF745
S11308C879FF02BD0020DFF8581309680968081881
S11308D8DFF84C13096849680818DFF844130968F5
S11308E889680818DFF838130968C9680818CC49F2
S11308F8096809690818CA49096849690818C84982
S1130908096889690818C6490968D1F8B810081827
S1130918002801D1012000E00020704780B5BF48BD
S1130928006810F1010F06D0BC4800F092F80028C6
S113093801D100200EE0B848006810F1010F06D07C
S1130948B54800F086F8002801D1002002E000F044
S11309587CF9012002BDB2480068704780B54FF4A5
S11309680072B1FBF2F303FB1213002B01D0002039
S11309780BE002688A4201D1012006E001604FF4CD
S11309880072001D00F094F9012002BD38B504007E
S11309980D00A248844208D19F4C29002000FFF78B
S11309A8DDFF002810D100200FE09D480068854233
S11309B803D19A4C9A480568EFE7200000F049F8FB
S11309C80028EAD1002000E0200032BD2DE9F041E2
S11309D804000F0015001E00780A4FF4007101FB93
S11309E800F8206810F1010F07D141462000FFF7F5
S11309F8B5FF002801D1002029E02068404508D02F
S1130A0841462000FFF7C2FF0400002C01D100205A
S1130A181DE02068381A0019071D00F05BF9201D35
S1130A28381AB0F5007F0AD318F500712000FFF7D3
S1130A38ADFF0400002C01D1002008E0271D287810
S1130A4838707F1C6D1C761E002EE6D10120BDE88F
S1130A58F081F8B505000124286800F079F8C0B2DF
S1130A68FF2801D100201DE0002600E0761C802E1E
S1130A7816D2286810EB860715EB860040680090AC
S1130A8800F028F9042200A93800FFF77DFE0028A9
S1130A9801D0002404E0386800998842E6D0002494
S1130AA82000C0B2F2BD5F480078C0B2472802D027
S1130AB8C0B2492802D14FF4007007E0C0B24828F8
S1130AC802D14FF4805001E04FF400607047F8B54C
S1130AD806000C00E4B2F6B2B44201D2002036E0BB
S1130AE84F48007AF6B2864205D34D4890F8B000D4
S1130AF8E4B2A04201D2002029E0FFF7D4FF0500A8
S1130B083000C0B200F04EF806002000C0B200F079
S1130B1849F807002000C0B200F061F8C019401E6F
S1130B28801B401CB0FBF5F4002700E07F1CBFB21B
S1130B38A4B2A7420AD200F0CDF8BFB205FB076001
S1130B48FFF726FE0028F1D0002000E00120F2BDC6
S1130B5838B50400002500E06D1CEDB20F2D1FD23E
S1130B6800F0B8F8EDB20C202D4900FB0510006820
S1130B788442F1D3EDB20C20294900FB051000682A
S1130B88EDB20C21264A01FB052149680818844264
S1130B98E2D2EDB20C20224900FB0510007A00E0F5
S1130BA8FF2032BD38B50400002500E06D1CEDB20D
S1130BB80F2D11D200F08EF8EDB20C20184900FB6D
S1130BC80510007AE4B2A042F0D1EDB20C20144929
S1130BD800FB0510006801E05FF0FF3032BD38B556
S1130BE80400002500E06D1CEDB20F2D11D200F0B9
S1130BF871F8EDB20C200A4900FB0510007AE4B242
S1130C08A042F0D1EDB20C20054900FB0510406864
S1130C1800E0002032BD0000780100207C030020A1
S1130C28081A0000FE81E00F1048006850F0010027
S1130C380E4908600E4841F6713101600B4800689E
S1130C48400840000949086070470848006850F0A7
S1130C58010006490860064800210160034800684D
S1130C6840084000014908607047000008000C4033
S1130C783C000C4080B500F02EF801BD10B500F022
S1130C883AF800280FD000F075F800F0C2F800F028
S1130C9836F8054908400549086000F030F844680A
S1130CA800F01BF8A04710BD80FFFF1F08ED00E00F
S1130CB870B504000D00160005E0287820706D1C3E
S1130CC8641C00F007F83000461E80B20028F4D1F6
S1130CD870BD7047704772B6704762B6704780B58A
S1130CE8FFF75AFD01BD80B5FFF764FD02BD80B56D
S1130CF8FFF78AFD02BD80B5FFF7E4FD02BD80B5AC
S1130D08FFF729FE02BD80B5FFF798FD002801D141
S1130D18002001E0FFF702FE02BD10B450F8041BE6
S1130D2881B102681218001D50F8043BDC0744BF67
S1130D38A9F10104E31852F8044B43F8044B091FC2
S1130D48F9D1EBE710BC704780B500F07FF800F0EC
S1130D58D1FA23480021017001BD80B5214800F073
S1130D6836FB012805D11E48002101701D4800F0FA
S1130D7897F801BD704780B5194A1278002A02D144
S1130D88C9B200F0F8FA00F085F801BD14480078FB
S1130D98002805D0022807D004D3032806D007E08A
S1130DA8402006E0002004E0002002E0002000E0EB
S1130DB8402080B270470A480078002805D00228ED
S1130DC807D004D3032806D007E0402006E000201B
S1130DD804E0002002E0002000E0402080B27047D8
S1130DE8740100201006002080B500F04AF802BD06
S1130DF880B500F00EF8114843F2AF610160104865
S1130E08002101600F48052101600F48002101609D
S1130E1801BD0C480021016070470A480068C003FE
S1130E2804D509480068401C07490860704780B524
S1130E38FFF7F3FF0448006802BD000014E000E077
S1130E4818E000E010E000E060060020DFF860042D
S1130E5800210170DFF8580400218164DFF8500490
S1130E68002180F84310DFF848040021A0F844105A
S1130E78DFF83C0400218170DFF83404002141705C
S1130E887047DFF82C040078002801D1002000E026
S1130E9801207047DFF81804002180F843107047D8
S1130EA880B50178FF291ED100F091F8DFF800041D
S1130EB890F84300012802D1102000F07EF8DFF8F2
S1130EC8F003B0F9440001280CDBDFF8E403012146
S1130ED880F84310DFF8D803B0F94410DFF8D403DE
S1130EE800F053F801BDDFF8C813097801294BD184
S1130EF80178C92932D0CC293FD0CF293AD0D0297A
S1130F082FD0D12933D0D2292ED0F32917D0F429C0
S1130F180FD0F5290AD0F6290ED0FA2912D0FC29C7
S1130F2813D0FD2914D0FE2915D029E000F0D2F8F9
S1130F38BCE700F0F1F8B9E700F0C1F8B6E700F053
S1130F4810F9B3E700F0A3F8B0E700F09AF8ADE7BA
S1130F5800F07FF8AAE700F06DF8A7E700F035F98C
S1130F68A4E700F054F9A1E700F012F99EE700F0B5
S1130F787FF99BE700F090F998E700F0A3F995E76B
S1130F88202000F01AF891E7ACE780B589B2FFF7A2
S1130F98F2FE01BD10B4002302E00478E318401CFB
S1130FA80C00611E002CF8D1DBB21360012010BCC8
S1130FB87047BF48002141707047BD49FE22CA707E
S1130FC8BB490871BA480221A0F84410704710B50B
S1130FD80400FFF7EEFFB64801210170B448FF2171
S1130FE8C170B34800210171B148007950F0100074
S1130FF8AF490871AE4800214171AD48AC494979FF
S11310084171FFF7C3FEAA498871FFF7D4FEA849C6
S1131018C871FFF7D0FE80B2000AA5490872A44837
S113102801214172A24801218172A1480821A0F836
S1131038441010BD10B504009D4800210170FFF74D
S1131048B8FF9B48FF21C17099480121A0F84410BA
S113105810BD9749FF22CA70954900220A71944924
S1131068934A52784A71924900228A71904900221F
S1131078CA718F4900220A728D490622A1F84420B8
S1131088704710B504000020FFF797FF10BD88498A
S1131098FF22CA708649884A8A64854900220A71EF
S11310A8834900224A71824900228A7180490722B1
S11310B8C1F807207E490822A1F8442070477C49DA
S11310C8FF22CA707A494068886479480121A0F8E7
S11310D84410704710B50400FFF758FE401E6178AD
S11310E8884203DA2220FFF768FF14E0627892B29C
S11310F86F48816C7148FFF7DBFD6D48FF21C170B3
S11311086B48806C61780818694988646078401C69
S11311186749A1F8440010BD10B50400FFF736FE76
S1131128401E6178884203DA2220FFF746FF17E061
S11311385F4861688164627892B25D48816C5F48F7
S1131148FFF7B6FD5A48FF21C1705948806C617891
S11311580818574988646078401C5549A1F8440028
S113116810BD80B55249FF22CA70554A416850489B
S1131178806CFFF70FFF4E4908714D4800214171FB
S11311884B48002181714A480821A0F8441001BD48
S113119810B504004648FF21C1704548002101717B
S11311A8434800214171FFF7F1FD414988714048E6
S11311B80021C1713E48002101723D48002141725D
S11311C83B480721A0F8441010BD10B50400FFF7F0
S11311D8DDFD621C80B2411E3548806CFFF783FD3B
S11311E8002803D13120FFF7E8FE0FE03048FF2143
S11311F8C170FFF7CBFD2E49896C80B2401E4018A0
S11312082B4988642A480121A0F8441010BD10B560
S11312180400FFF7BBFD801E6178884203DA2220B0
S1131228FFF7CBFE23E02248FF21C17020480121AB
S1131238A0F844106078002807D1FFF764FD00285F
S113124802D13120FFF7B9FE11E0A21C61781848D9
S1131258806CFFF748FD002803D13120FFF7ADFE6D
S113126805E01348806C617808181149886410BD3A
S113127880B541680E48806CFFF739FD002803D11A
S11312883120FFF79AFE06E00948FF21C17008489B
S11312980121A0F8441001BD10B50400FFF7EEFCCD
S11312A80348FF21C17002480121A0F8441010BD71
S11312B88005002083050020081C00008405002008
S11312C88705002080B53120FFF777FE01BD50F86F
S11312D8041B61B150F8042BD30744BFA9F10103DF
S11312E89A18002342F8043B091FFAD1EFE7704724
S11312F84163704700B585B000A86949102200F021
S1131308EDF801216748FFF702F8012304220621BA
S1131318022000F020F9002301220721022000F016
S11313281AF901216048FEF7F2FF02215F48FFF72E
S1131338F2F801215E48FEF747FF01215C48FEF7F9
S1131348E6FF00208DF8000000A95A4800F0B7F91C
S11313584FF416520021574800F06FF956480321FC
S1131368016004215348FFF7C3FF0521514800F0E9
S11313788BF905B000BD70B504000D00EDB2412D28
S113138803DB6C214D4800F0D1F92800C0B200F00D
S113139872F8C0B2012803D07021484800F0C6F999
S11313A800260DE0FFF796FCB6B2305D00F063F856
S11313B8C0B2012803D07921404800F0B7F9761C5F
S11313C82800C0B2B6B280B28642EBD370BD10B565
S11313D804003B480078002813D13A4800F03DF84F
S11313E8012838D137480078002834D0FFF71FFD8A
S11313F835490860354800210170314801210170E0
S113140829E0324800782F494018401C00F025F89C
S1131418012816D12D480078401C2C4908702B4807
S1131428007828490978884215D12848027892B268
S113143827492000FFF73CFC2148002101700120C6
S11314480AE0FFF7F4FC204909686431814202D2BA
S11314581B4800210170002010BD10B504000020B5
S11314681C490968490704D5124800F04BF9207053
S11314780120C0B210BD80B517490968C90601D456
S113148800200CE00100C9B20A4800F041F901E06B
S1131498FFF720FC10480068C006F9D5012002BDFA
S11314A8DC1B000000C20200002304000300120039
S11314B8401516000044084054440840001B00002E
S11314C86C060020CC050020640600206B06002072
S11314D8CD0500202C44084008440840103A07D39E
S11314E830B4B1E83810103AA0E83810F9D230BC5A
S11314F8530724BFB1E80810A0E8081044BF51F806
S1131508043B40F8043BD20724BF31F8022B20F8EF
S1131518022B44BF0B7803707047083A07D3B1E82D
S11315280810083A40F8043B40F804CBF7D25307B4
S1131538E4E70000C0B224223B4B02FB00321268ED
S113154892089200C9B21143C0B22422364B02FB5E
S113155800300160704770B4D2B2002A12D0002B58
S113156808D0C0B22424304D04FB005401258D401A
S1131578256107E0C0B224242B4D04FB0054012547
S11315888D406561082919D2C0B22424264D04FB74
S1131598005464680F250E00F6B2B600B540AC439B
S11315A8D2B20D00EDB2AD0012FA05F52C43C0B26B
S11315B824251D4E05FB00656C601AE0C0B2242486
S11315C8194D04FB0054A4680F250E00083EF6B21A
S11315D8B600B540AC43D2B20D00083DEDB2AD0043
S11315E812FA05F52C43C0B224250F4E05FB0065FD
S11315F8AC60D2B2002A14D1002B09D0C0B2242284
S1131608094B02FB0030012212FA01F1016108E0E2
S1131618C0B22422044B02FB0030012212FA01F169
S1131628416170BC7047000000600040026CD20742
S113163802D4426C0A42FCD1704738B50400150044
S1131648002906D10C4884420ED10C48FEF793FEBB
S113165801004801B0FBF5F5203DED000421200010
S1131668FFF7E4FFE56031BD0548844201D1054830
S1131678ECE7F8E7000000000040084040051400CB
S1131688004408404015160038B50400C9B2CD43DB
S113169815F005056D00C9B20D4302212000FFF7BE
S11316A8C5FF656031BDC9B2002905D0416C002968
S11316B8FCD10121016401E000210164704738B5BF
S11316C804000D0002212000FFF7B0FF0A2060602B
S11316D801212000FFF7E7FF206830F01C00297B78
S11316E80843697B0843A97B08432060AA686968A2
S11316F82000FFF7A2FF2878606000212000FFF790
S1131708D2FF31BD81688906FCD5C069C0B2704773
S113171838B504000D00A068C006FCD5402120009F
S1131728FFF784FFEDB2A56231BD000080B5034A1E
S1131738106003480160FFF7CDFAFCE7500600206B
S11317485406002080B568480168080E00280DD1A9
S11317586648026832F07002026065480268D20086
S1131768D2080260026872F060620260080E0428FF
S113177813D25F48016831F4FC5101605D480021CF
S113178801605D48002101605C48002101605C48FB
S1131798002101605B480021016000A800F0DCF82A
S11317A89DF80000012811D19DF80100002804D1FA
S11317B85048016851F0020101609DF801000228B7
S11317C804DA4D48016851F0010101604E4801688E
S11317D84E48814224D24848016851F4904101603E
S11317E84B480068000410F0FE414948006810F0B6
S11317F87F0051EA00414648006810F4FE40014366
S11318084348006810F07F000143424801604248A1
S11318184249096801603848016831F4904101601F
S113182801BD80B500F005F800F0ACF800F0B8F898
S1131838FCE780B5FEF77EFFFFF784FF0122012154
S11318480020FEF7CCFE2B48006850F00F00294911
S113185808602948006840F47F4050F0FF0026499A
S1131868086000212E48FEF752FD00212D48FEF79E
S11318784EFD00212C48FEF74AFD00212B48FEF7B7
S113188846FD00212A48FEF742FD00212948FEF7BB
S11318983EFD00212848FEF73AFD00212748FEF7BF
S11318A836FD00212648FEF732FD00212548FEF7C3
S11318B82EFD00212448FEF72AFD00212348FEF7C7
S11318C826FD00212248FEF722FD00212148FEF7CB
S11318D81EFD0123052209210120FFF73CFE0221F8
S11318E80120FFF727FE01BDFC81E00F0CA00C408E
S11318F820600C4040800C4044800C4058800C40D0
S113190860800C4078800C40F081E00F00BA8A4C6B
S1131918B481E00F342000402C400040C881E00F1F
S113192800030400001304000033040000A20200B2
S1131938000202000012020000220200003202002B
S1131948007202000082020000B2020000E20200FB
S113195800F2020000D202000749096811F03F01B1
S113196801700649096811F0F001054A1268C2F3CA
S11319780312114341707047E0FF0FE0E8FF0FE0E6
S1131988ECFF0FE080B5FFF775F9FFF7A2F9FFF751
S11319982FFAFFF7A4F9FFF7D7F900F00BF801BD08
S11319A880B5FFF797F9FFF738FAFFF7D6F900F093
S11319B80CF801BD80B5104801210170FFF737FA12
S11319C80E49086000F001F801BD80B5FFF70CFA74
S11319D8012810D00848007801280CD1FFF727FA0D
S11319E80649096811F5FA71884204D302480021AE
S11319F80170FFF743F901BD6A060020580600206C
S1131A080020000000200000010000000040000049
S1131A180020000002000000006000000020000018
S1131A280300000000800000002000000400000003
S1131A3800A00000002000000500000000C0000015
S1131A48002000000600000000E000000020000064
S1131A58070000000000010000200000080000004A
S1131A6800200100002000000900000000400100DF
S1131A78002000000A0000000060010000200000AF
S1131A880B00000000800100002000000C00000092
S1131A9800A00100002000000D00000000C00100AB
S1131AA8002000000E00000000E0010000200000FB
S1131AB80F000000433A5C576F726B5C736F667477
S1131AC8776172655C4F70656E424C545C54617208
S1131AD86765745C536F757263655C41524D434D21
S1131AE8335F45464D33325C4941525C76656374D5
S1131AF86F72732E63000000433A5C576F726B5C1D
S1131B08736F6674776172655C4F70656E424C548E
S1131B185C5461726765745C536F757263655C418C
S1131B28524D434D335F45464D33325C7561727493
S1131B382E63000010B5074979441831064C7C44DB
S1131B48163404E00A68081D511888470146A14262
S1131B58F8D110BD080000002800000073F7FFFF4B
S1131B68F80400007801002000000000AFF1FFFF36
S1131B78780100009400000000000020000000002C
S1131B8800F009F8002801D0FFF7D4FF0020FFF780
S1131B9848FE00F002F80120704700F001B8000088
S1131BA80746384600F002F8FBE7000080B5C04657
S1131BB8C046024A11001820ABBEFBE7260002000B
S1131BC8034B9D46C046C046C046C046FFF7D8FFF3
S1131BD870070020050000000000000080250000B8
S1131BE80000000080B53C210148FFF79FFD01BDBE
S1131BF8BC1A0000C046C046C046C046FFF7C0FF36
S1131C084F70656E424C54005449554A126852F05C
S1131C180102534B1A60534A106053480122026070
S1131C2852480068400708D54D48006840084000FD
S1131C384B4908605FF0FF3029E04C480068800792
S1131C4808D54748006840084000454908607FF0C7
S1131C5801001CE044480222026000E0491E434897
S1131C680068C00701D50029F8D1002908D13C48EB
S1131C780068400840003A4908607FF0020006E026
S1131C88374800684008400035490860002070471C
S1131C9830B4334B1B6853F00103314C2360931069
S1131CA8002200E0521C9A424FDA10EB82042D4DB8
S1131CB82C602D4C012525602C4C2468640708D51C
S1131CC82748006840084000254908605FF0FF3055
S1131CD842E0264C2468A40708D521480068400837
S1131CE840001F4908607FF0010035E01B4C00E00C
S1131CF8641E1E4D2D682D0701D4002CF8D1002C2C
S1131D0808D11748006840084000154908607FF06A
S1131D18020021E051F82240154D2C60124C082590
S1131D2825600E4C00E0641E104D2D68ED0701D5AA
S1131D38002CF8D1002CB5D10948006840084000AF
S1131D48074908607FF0020006E00548006840087B
S1131D58400003490860002030BC70478096980012
S1131D6808000C4010000C400C000C401C000C40F7
S1131D7818000C400048E80100800000040000003E
S9031BFDE4
